:100E5A0000C000F900A400B000990092008200F8D6
:100E6A00008000900088008300C600A10086008EE2
:05108200E52F5401FF01
:0A108700E51125E0F511EF421122FA
:0D10CA00E51125E0F511EFF454014211226B
:100F19001313135401FD1200031210F17861E65402
:020F290001FFC6
:040F2B00EF5211224E
:07115D00EFF45401521122CE
:04119A00EF421122ED
:07116400EFF45401421122D7
:0E10A000E511F45401FFE51154FE4FF5112245
:06118E00E5115401FF22EF
:0D10D700E511C313FFE51154015FF511226F
:0D10E400E511C313FFE51154014FF5112272
:050F6F0013135401FD05
:0E0F7400E51125E0F511EDF45F540142112264
:0E10AE00E51125E0F511EFF45D540142112229
:08000300EDF45F5401521122DB
:08114500EFF45D540152112288
:08114D00EDF45F540142112290
:08115500EFF45D540142112288
:07116B00EDF45F5401FF22C7
:07117200EFF45D5401FF22C0
:0D10F100E51825E0FFE51154014FF5182228
:0D10FE00E5185401FFE51154FE4FF51122D5
:100F8200E5185401FFE51154FE4FF511E518C3139E
:030F9200F518222D
:101072008E528F53E5532DFFE5523C8FF0020A7FCB
:100F95008E528F53C3E5539DFFE5529C8FF0020A95
:010FA5007FCC
:100E7A0090010CE0FEA3E0FF7B017A01790C7D0A68
:020E8A007C00EA
:090E8C001209BEEE8FF0020A7F8C
:0F1091008B528A5389541209D0EE8FF0020A7FD6
:07117900E475F001020A47D2
:0711800074FFF5F0020A47BD
:100FA6008E5B8F5CE55B5CFFE55C5DCF8FF0020AD4
:010FB6007FBB
:100FB7008E5D8F5EE55D4CFFE55E4DCF8FF0020ADB
:010FC7007FAA
:100FC8008E5F8F60E55F6CFFE5606DCF8FF0020A82
:010FD8007F99
:100FD900EFF4FFEEF4FEEF2401FFE43E8FF0020A86
:010FE9007F88
:06119400EFF45401FF22FC
:0E0F5B0090010CE0FEA3E0FF7B017A01790E0D
:060F6900EE8FF0020A7F8A
:0A113B00EFF4FFEEF48FF0020A7FDC
:100E04008B4B8A4C894D120A1CFFAEF0AB4EAA4F95
:100E1400A950120A1CFDAB4BAA4CA94DE5F08DF06C
:0F0E2400120A7FAB4EAA4FA950EE8FF0020A7F41
:100AF3008E528F538B548A5589567C037DE8120995
:100B0300D0EFC454F07B00FAAE52AF537C037DE8C0
:100B13001209D08C528D53AE52AF537C007D6412B8
:100B230009D0EFFEE4EE4202AE52AF537C007D6487
:100B33001209D08C528D53AE52AF537C007D0A12F2
:100B430009D0EFC4F8540FC868FFEEC454F048FE50
:100B5300EFFBEE4202AE52AF537C007D0A1209D086
:100B63008C528D53E5524AFFE5534BAB54AA55A91A
:070B730056CF8FF0020A7F4C
:100BF9008E578F58E558780CCEA2E713CE13D8F844
:100C09007E00540FFF7C037DE81209BE8E598F5A6E
:100C1900E557FF3395E07E00EF540FFF7C007D64BC
:100C29001209BEEF255AF55AEE3559F559E558AE70
:100C3900577804CEA2E713CE13D8F87E00540FFFDD
:100C49007C007D0A1209BEEF255AF55AEE3559F591
:100C590059E558540F255AF55AE43559F559855A25
:040C6900F0020A7F0C
:100E9500E51125E0F511C3EF9DEC6480F8EE648063
:0B0EA500984004431101225311FE226B
:100EB000E51125E0F511D3EF9DEC6480F8EE648038
:0B0EC000985004431101225311FE2240
:100ECB00E51125E0F511D3EF9DEC6480F8EE64801D
:0B0EDB00984004431101225311FE2235
:100EE600E51125E0F511C3EF9DEC6480F8EE648012
:0B0EF600985004431101225311FE220A
:100F2F00E51125E0F511EF6D7002EE6C60044311D1
:060F3F0001225311FE2205
:100F4500E51125E0F511EFB50508EEB504044311EB
:060F550001225311FE22EF
:100FEA00C3EF9DEC6480F8EE64809850035311FEC1
:010FFA0022D4
:100FFB00D3EF9DEC6480F8EE64809840035311FEB0
:01100B0022C2
:10100C00D3EF9DEC6480F8EE64809850035311FE8E
:01101C0022B1
:10101D00C3EF9DEC6480F8EE64809840035311FE9D
:01102D0022A0
:0C110B00EFB50507EEB504035311FE22FA
:0C0F0100900110E0FEA3E0FF7D017C00E9
:0C0F0D00EF6D7002EE6C60035311FE22C9
:10102E00C3EF9DEC6480F8EE648098400343110199
:01103E00228F
:10103F00D3EF9DEC6480F8EE648098500343110168
:01104F00227E
:10105000D3EF9DEC6480F8EE648098400343110167
:01106000226D
:10106100C3EF9DEC6480F8EE648098500343110156
:01107100225C
:0C111700EF6D7002EE6C600343110122CA
:0C112300EFB50507EEB5040343110122EF
:07118700E4FF0FBF0AFC2288
:100DD400E4FEC2B4121187C2B3121187D2B3121146
:100DE40087D2B4121187E4FDEE25E0FE309403436C
:100DF4000601C2B3121187D2B30DBD08EBAF0622B0
:1007DD000510E510C394054003E4F510E510146011
:1007ED005B1470030208991470030208E52403607A
:1007FD00030209377C0090000DE0540FFD25E0FF4A
:10080D00EC33FE745A2FF582740E3EF583E493FC9F
:10081D00740193FD43040890010AE0FFC413131300
:10082D00540130E0057DFF02098DEF131313541FA2
:10083D0020E00302098D53057F02098D90000CE025
:10084D00FEA3E07804CEA2E713CE13D8F87C0054B3
:10085D000FFD25E0FFEC33FE745A2FF582740E3E2A
:10086D00F583E493FC740193FD43040490010BE0C4
:10087D0030E0057DFF02098D90010AE0FFC4540FA1
:10088D0020E00302098D53057F02098D90000CE0D5
:10089D00FF3395E07C00EF540FFD25E0FFEC33FEB8
:1008AD00745A2FF582740E3EF583E493FC74019314
:1008BD00FD43040290010BE0FFC31330E0057DFF03
:1008CD0002098D90010AE0FFC413540720E00302D2
:1008DD00098D53057F02098D90000CE0FEA3E07891
:1008ED000CCEA2E713CE13D8F87C00540FFD25E0F3
:1008FD00FFEC33FE745A2FF582740E3EF583E493AC
:10090D00FC740193FD43040190010BE0FF1313549C
:10091D003F30E0047DFF806890010AE0FFC41313AF
:10092D00540330E05B53057F805690010BE0F9C412
:10093D001313540175F008A4FBAAF0E9C4131313A3
:10094D00540175F010A4FFE5F04AFAEF4BFBE9C432
:10095D0013540175F004A4FFEA45F0FAEB4FFBE9DF
:10096D00C4540125E0FFE4334AFEEB4FFFE91313B6
:10097D00135401FBEEEF4BF4FFEEF47410FCAD07D6
:10098D007B10C2B3121187EC20E704C2B78002D2EC
:10099D00B7121187ED25E0FDEC33FCD2B3121187B0
:1009AD00DBE0D2B7121187C2B5121187D2B5021191
:0109BD0087B2
:1005F700E52E70030207DC152E0517E517B405175E
:10060700AF30EFC4135401F45401FFC43354E0FF77
:10061700E53054DF4FF530E517B40A1CAF30EFC4AF
:10062700135401F45401FFC43354E0FFE53054DFA1
:100637004FF530051DE4F517E4F552E55213131392
:10064700541F2412F8E6FD7C00E5525407FF74019D
:100657007E00A807088005C333CE33CED8F9FFEE56
:100667005CFEEF5D4E6043E55225E025E0246EF524
:1006770082E43400F583E0FEA3E0FFE55225E025A0
:10068700E0246CF582E43400F583E0FCA3E0C39F2B
:10069700EC9E5016E55225E025E0246CF582E43403
:1006A70000F583E475F001120A06E55225E025E01E
:1006B700246EF582E43400F583E0FEA3E0FFE55203
:1006C70025E025E0246CF582E43400F583E0FCA303
:1006D700E0C39FEC9E407AE55225E025E0246CF5C7
:1006E70082E43400FEC3E582946CFFEE9400FE7C46
:1006F700007D021209D07C007D021209D07C007DAA
:10070700081209D0741E2FF8C000E6FFC007E55293
:1007170025E025E0246CF582E43400FEC3E58294ED
:100727006CFFEE9400FE7C007D021209D07C007DF8
:10073700021209D07C007D081209D0AF057401A808
:1007470007088002C333D8FCFED0E04ED000F68005
:1007570079E55225E025E0246CF582E43400FEC3F8
:10076700E582946CFFEE9400FE7C007D021209D0B6
:100777007C007D021209D07C007D081209D0741E0E
:100787002FF8C000E6FFC007E55225E025E0246CFE
:10079700F582E43400FEC3E582946CFFEE9400FE1C
:1007A7007C007D021209D07C007D021209D07C00FA
:1007B7007D081209D0AF057401A807088002C3336A
:1007C700D8FCF4FED0E05ED000F60552E552642076
:0607D7006003020642224D
:100D1A00E51DB41E19AF30EFC413135401F4540186
:100D2A00FFC4333354C0FFE53054BF4FF530E51DDF
:100D3A00B43C1CAF30EFC413135401F45401FFC484
:100D4A00333354C0FFE53054BF4FF530E4F51D226C
:03000B00020C6D77
:100C6D00C0E0C0D075D008758CEEAF30EF13131304
:100C7D005401F45401FF33333354F8FFE53054F786
:100C8D004FF530053AE53A30E0020516E53AB40A7B
:100C9D0015AF30EFC45401F45401FFC454F0FFE517
:100CAD003054EF4FF530E53AB4141AAF30EFC45469
:100CBD0001F45401FFC454F0FFE53054EF4FF5300B
:0A0CCD00052E753A00D0D0D0E032B9
:100CD7007594FF752F05E4F530F53190000CF0A3FE
:100CE700F090010BE054F7F054EFF054DFF054BFED
:100CF700F0547FF090010AE054F7F054EFF054DF1E
:100D0700F054BFF0547FF0A3E054FEF054FDF054CC
:030D1700FBF022CC
:04119E00752F09227E
:100D5A00E4FFEF25E025E0246CF582E43400F58316
:100D6A00E4F0A3F00FBF20EAE4FF7F4090002CE4F8
:100D7A00F0A3DFFCE4FF741E2FF8E4F60FBF04F6BD
:0D0D8A00E4FF74192FF8E4F60FBF04F62201
:0E10BC00758911D2B4D2B9D2A9D28CD2AF228A
:100D9700AFA0EFC3135455FEEF25E054AA4EFF133F
:100DA700135433FEEF25E025E054CC4EFF54F0FEFC
:100DB700E590540F4EF4F522EF540FF4540FF5233A
:0D0DC700120DD4EFF4F5248528800207DD1D
:100B7A00E4FF74222FF8E6FE743F2FF8A6060FBF93
:100B8A0006F0E4FF74282FF8E6FE74452FF8A6064F
:100B9A000FBF06F0E4FF74612FF8E6FE74202FF50C
:100BAA0082E43401F583EEF00FBF20EAE4FF74EC2F
:100BBA002FF582E43400F583E0FE74402FF582E4D9
:100BCA003401F583EEF00FBF20E4E4FF741E2FF822
:100BDA00E6FE74362FF8A6060FBF04F0E4FF741978
:0F0BEA002FF8E6FE74322FF8A6060FBF04F02294
:100E3300755101120CD7120D5A1210BC120D9712D4
:100E4300000E1205F7120D1A120B7AE55160EDE44C
:070E5300F55112119E80E52C
:10000E00AF2FEF13135401FF121087E5245401FF95
:10001E00E5415401FD12114DE51130E007E4900168
:10002E000CF0A3F0E51130E007E490010EF0A3F020
:10003E00E51130E007E4900110F0A3F0E51130E097
:10004E00067861E654FEF6121082E51130E00F904C
:10005E00010CE0FEA3E0FF7DE77C0312101D1210E1
:10006E00F1E5225401FFE53F120F1CE51130E007C8
:10007E00E490010CF0A3F0E51130E0067861E6544F
:10008E00FEF6120F82E51130E003120E7A1210FE08
:10009E00AF22EFC3135401FFAE3FEEC3120F1BE5A9
:1000AE001130E007E490010CF0A3F0E51130E0060A
:1000BE007861E654FEF6120F82E51130E003120E5F
:1000CE007AE51130E01590010CE0FEA3E0FF7B0114
:1000DE007A01790C7D017C001210721210FEAF2293
:1000EE00EF13135401FFAE3FEE120F1AE51130E07D
:1000FE0007E490010CF0A3F0E51130E0067861E61C
:10010E0054FEF6120F82E51130E003120E7AE5115D
:10011E0030E01590010CE0FEA3E0FF7B017A01793F
:10012E000C7D027C001210721210FEAF22EF131320
:10013E00135401FFAE3FEE120F19E51130E007E444
:10014E0090010CF0A3F0E51130E0067861E654FE64
:10015E00F6120F82E51130E003120E7AE51130E04F
:10016E001590010CE0FEA3E0FF7B017A01790C7D76
:10017E00037C001210721210FEAF22EFC45401FF66
:10018E00AE3FEEC4120F1CE51130E007E490010CF7
:10019E00F0A3F0E51130E0067861E654FEF6120F9A
:1001AE0082E51130E003120E7AE51130E015900170
:1001BE000CE0FEA3E0FF7B017A01790C7D047C004C
:1001CE001210721210FEAF22EFC4135401FFAE3F95
:1001DE00EEC4120F1BE51130E007E490010CF0A302
:1001EE00F0E51130E0067861E654FEF6120F82E576
:1001FE001130E003120E7AE51130E01590010CE09B
:10020E00FEA3E0FF7B017A01790C7D057C001210C4
:10021E00721210FEAF22EFC413135401FFAE3FEE65
:10022E00C4120F1AE51130E007E490010CF0A3F0B0
:10023E00E51130E0067861E654FEF6120F82E51104
:10024E0030E003120E7AE51130E01590010CE0FE5D
:10025E00A3E0FF7B017A01790C7D067C00121072FF
:05026E001210FEAF229A
:10027300EFC41313135401FFAE3FEEC4120F19E57D
:100283001130E007E490010CF0A3F0E51130E00633
:100293007861E654FEF6120F82E51130E003120E88
:1002A3007AE51130E01590010CE0FEA3E0FF7B013D
:1002B3007A01790C7D077C001210721210FEE5237F
:1002C3005401FFE540120F1CE51130E007E49001F3
:1002D3000CF0A3F0E51130E0067861E654FEF61267
:1002E3000F82E51130E003120E7AE51130E015902C
:1002F300010CE0FEA3E0FF7B017A01790C7D087C11
:1003030000121072120F82AF23EFC3135401FFAE1A
:1003130040EEC3120F1BE51130E007E490010CF02F
:10032300A3F0E51130E0067861E654FEF6120F8281
:10033300E51130E003120E7AE51130E01590010C5F
:10034300E0FEA3E0FF7B017A01790C7D097C0012BA
:100353001072AF24EFC4135401FFAE41EEC4120F69
:1003630070E51130E00D7B017A0179107F017E0089
:10037300120F69E51130E003120F5BE51130E0065F
:100383007861E64401F6AF24EF13135401FFAE4145
:10039300EE120F6FE51130E00D7B017A0179107FCA
:1003A300027E00120F69E51130E003120F5BE511C5
:1003B30030E0067861E64401F6AF24EFC45401FF50
:1003C300AE41EEC45401FD120F74E51130E00D7B14
:1003D300017A0179107F037E00120F69E51130E085
:1003E30003120F5BE51130E0067861E64401F6AFD6
:1003F30024EF1313135401FFAE41EE13120F6FE5F5
:100403001130E00D7B017A0179107F047E00120F19
:1004130069E51130E003120F5BE51130E006786106
:10042300E64401F61210821210F1E51130E00312D6
:100433000F0112118EEF5401FF33333354F8FF9041
:10044300010BE054F74FF01210FEE51130E00F906E
:100453000110E0FEA3E0FF7D027C00120F0D1211DC
:100463008EEF5401FFC454F0FF90010BE054EF4FA3
:10047300F01210FEE51130E00F900110E0FEA3E052
:10048300FF7D037C00120F0D12118EEF5401FFC488
:100493003354E0FF90010BE054DF4FF0120F82E57D
:1004A3001130E00F900110E0FEA3E0FF7D047C001B
:1004B300120F0D12118EEF5401FFC4333354C0FFDA
:1004C30090010BE054BF4FF0AF24EFC3135401FF6F
:1004D300AE41EEC3120F701210F1E51130E00312BA
:1004E3000F01E51130E01990010EE0FEA3E0FF904B
:1004F300010CE0FCA3E0FD7B017A01790C12107280
:100503001210FEE51130E00F900110E0FEA3E0FFB2
:100513007D027C00120F0DE51130E01990010EE011
:10052300FEA3E0FF90010CE0FCA3E0FD7B017A0158
:10053300790C120F951210FEE51130E00F900110A7
:10054300E0FEA3E0FF7D037C00120F0DE51130E018
:100553001990010EE0FEA3E0FF90010CE0FCA3E084
:10056300FD7B017A01790C120E8C1210FEE511301D
:10057300E00F900110E0FEA3E0FF7D047C00120F6A
:100583000DE51130E01990010EE0FEA3E0FF9001AC
:100593000CE0FCA3E0FD7B017A01790C12109112AF
:1005A3000F82E51130E007E4900110F0A3F0121080
:1005B30082E51130E00F90010CE0FEA3E0FF7D0F18
:1005C3007C2712100C12118EEF5401FFC433333306
:1005D3005480FF90010BE0547F4FF0121082E5111D
:1005E30030E00FA3E0FEA3E0FF7B017A00790C1259
:0405F3000AF30022E5
:0300000002112FBB
:0C112F00787FE4F6D8FD758180020E3355
:1009BE00EF8DF0A4A8F0CF8CF0A428CE8DF0A42E4D
:0209CE00FE2207
:1009D000C2D5EC30E709B2D5E4C39DFDE49CFCEE42
:1009E00030E715B2D5E4C39FFFE49EFE120A9EC312
:1009F000E49DFDE49CFC8003120A9E30D507C3E40D
:060A00009FFFE49EFE22B0
:100A0600C5F0F8A3E028F0C5F0F8E582158270027B
:060A16001583E038F02218
:100A1C00BB010A89828A83E0F5F0A3E022500687A5
:100A2C00F009E71922BBFE07E3F5F009E319228967
:0B0A3C00828A83E493F5F0740193229A
:100A4700BB010789828A83020A06500B09C5F02772
:100A5700F7C5F01937F722BBFE0D09F8E325F0F3C8
:100A6700C5F019E338F322F889828A837401932544
:080A7700F0C5F0F8E493382209
:100A7F00BB010A89828A83F0E5F0A3F0225006F7C2
:0F0A8F0009A7F01922BBFE06F3E5F009F31922BF
:100A9E00BC000BBE0029EF8DF084FFADF022E4CC3C
:100AAE00F875F008EF2FFFEE33FEEC33FCEE9DEC05
:100ABE00984005FCEE9DFE0FD5F0E9E4CEFD22ED4B
:100ACE00F8F5F0EE8420D21CFEADF075F008EF2F95
:100ADE00FFED33FD4007985006D5F0F222C398FD86
:050AEE000FD5F0EA2223
:00000001FF
